:100000004F0A2E0047090E022C000A066C000F0949
:1000100043064B0A0F0943064B0A0F094B0A0E020F
:10002000AC01010C2A006B0000024E018C01430759
:100030000008AA024306EB03140A0008240060002B
:10004000A40284061F0A4B0A6D002C00FF0CEC0171
:100050000307ED0103074B0A030C2B00DF0C3209E9
:10006000260A6B002A00E70CEA016B02FC0C03076E
:100070003D0AEA010306390AEA010000EB03390AE6
:100080000A06420A2A07460A0000460A0008070133
:10009000270006004B0AC404A40400000008640002
:1000A000FF0C27002900A90409020200100C1E09F8
:1000B000010C3100040C910003066C0A260527048C
:1000C00007020600C80C24092604270407020600BC
:1000D000C80C2409F1035A0A010C2A00060C24005A
:1000E000080C01090A0230000F0C2409320C9000A0
:1000F00003067B0A580A14024306010C430740001A
:100100002F004C0C900040000306010C4F012F0003
:100110007D0C9000010C030640004F014306920A3B
:10012000010C3400010C94004306010C430740000D
:100130002F00B00C900040000306010C4F012F006F
:10014000E10C9000010C030640004F014306AA0A8F
:10015000020C3400020C94004306010C43074000DB
:100160002F004C0C900040000306010C4F012F00A3
:100170007D0C9000010C030640004F014306C20AAB
:10018000030C3400030C94004306010C43074000A9
:100190002F004C0C900040000306010C4F012F0073
:1001A0007D0C9000010C030640004F014306D90A64
:1001B000200B030C94004306010C430740002F0062
:1001C000B00C900040000306010C4F012F00E10C21
:1001D0009000010C030640004F014306F00A2F0B6C
:1001E000040C94004306010C430740002F004C0C04
:1001F000900040000306010C4F012F007D0C900081
:10020000010C030640004F014306080B030C3400A9
:10021000040C94004306010C430740002F00B00C6F
:10022000900040000306010C4F012F00E10C9000EC
:10023000010C030640004F0143061F0B200B6C0A04
:10024000B2024306B302030C930003072E0B4307CD
:100250002D0B850C920003072E0B2F0B6C0A460406
:100260004704070206002605270407020600FA0CC9
:100270002409470507020600260427040702060092
:1002800073007200040C34000B0C2D00B80C25090F
:020290006C0AF6
:0203FE000000FD
:021FFE00EA0FE8
:00000001FF
